:100000000C949D030C94E4030C94E4030C94E4031B
:100010000C94E4030C94E4030C94E4030C94E403C4
:100020000C94E4030C94E4030C941C220C94D8214B
:100030000C94D7280C94E4030C94E4030C94E4038C
:100040000C94E4030C94E4030C94E4030C94E40394
:100050000C94E4030C94B3280C94E4030C94E40390
:100060000C94E4030C94E4030C94E4030C94E40374
:100070000C94E4030C94E4030C94E4030C94E40364
:100080000C94E4030C94E4030C94E4030C94E40354
:100090000C94E4030C94E4030C94E4030C94E40344
:1000A0000C94E4030C94E4030C94E40305010902AA
:1000B000A10185020901A100050919012905150001
:1000C00025019505750181029501750381010501E1
:1000D000093009311581257F950275088106093897
:1000E0001581257F950175088106050C0A380215D2
:1000F00081257F950175088106C0C005010980A191
:1001000001850319012AB700150126B7009501756D
:10011000108100C0050C0901A101850419012AA064
:1001200002150126A002950175108100C005010984
:1001300006A1018505050719E029E71500250195A8
:1001400008750181020507190029EF1500250195A1
:10015000F0750181020508190129059505750191C0
:1001600002950175039101C00660FF0961A10109B3
:1001700062150026FF0095207508810209631500AD
:1001800026FF00952075089102C005010906A1010E
:10019000050719E029E71500250195087501810279
:1001A0009501750881010507190029FF150026FF33
:1001B0000095067508810005081901290595057542
:1001C000019102950175039101C00000000000003B
:1001D000000000000000000000000000000000001F
:1001E00000000000000000000000000000007E0F82
:1001F00000D4FFFFFFC700000078000000000000EF
:1002000000002A2B28000000000000000000000071
:10021000000000000029000000002C1E34202122D4
:1002200024342627252E362D3738271E1F2021223D
:10023000232425263333362E37381F0405060708B6
:10024000090A0B0C0D0E0F101112131415161718A6
:10025000191A1B1C1D2F3130232D350405060708E4
:10026000090A0B0C0D0E0F10111213141516171886
:10027000191A1B1C1D2F3130354C000101010101E1
:10028000010101010202020202020202020303034F
:10029000030303030304040404040404050505051F
:1002A00005060606060607070707070808080809DF
:1002B0000909090A0A0A0B0B0B0C0C0C0D0D0D0E8B
:1002C0000E0E0F0F0F101011111112121313141420
:1002D000151516161717181819191A1A1B1B1C1D95
:1002E0001D1E1E1F202021222223242425262627EE
:1002F0002829292A2B2C2D2D2E2F30313232333420
:1003000035363738393A3B3C3D3E3F404142434425
:1003100045464748494A4C4D4E4F50515354555607
:1003200058595A5B5D5E5F616264656668696B6CB3
:100330006D6F7072737577787A7B7D7E808283852E
:1003400087888A8C8E8F91939596989A9C9EA0A26E
:10035000A3A5A7A9ABADAFB1B3B5B7BABCBEC0C278
:10036000C4C6C9CBCDCFD1D4D6D8DBDDDFE2E4E73C
:10037000E9EBEEF0F3F5F8FAFDFFFFAA7F55402216
:1003800023252628292A2C2D2F3032333536383A8A
:100390003B3D3E4042434547494A4C4E50515355E0
:1003A00057595A5C5E6062646668696B6D6F717301
:1003B0007577797B7D7F81838587898A8C8E909202
:1003C0009496989A9C9E9FA1A3A5A7A8AAACAEAF0D
:1003D000B1B3B4B6B8B9BBBCBEBFC1C2C3C5C6C752
:1003E000C9CACBCCCDCED0D1D2D2D3D4D5D6D7D703
:1003F000D8D9D9DADADBDBDBDCDCDCDCDCDDDDDD4B
:10040000DDDCDCDCDCDCDBDBDBDADAD9D9D8D7D746
:10041000D6D5D4D3D2D2D1D0CECDCCCBCAC9C7C6F3
:10042000C5C3C2C1BFBEBCBBB9B8B6B4B3B1AFAE31
:10043000ACAAA8A7A5A3A19F9E9C9A9896949290D7
:100440008E8C8A89878583817F7D7B7977757371AF
:100450006F6D6B6968666462605E5C5A595755538C
:1004600051504E4C4A4947454342403E3D3B3A3845
:1004700036353332302F2D2C2A29282625232229C0
:10048000003A003B003C003D003E003F0040004180
:100490000042004300440045000151490035001E60
:1004A000001F002000210022002300240025002638
:1004B0000027002D002E002A0035002B0014001A02
:1004C000000800150017001C0018000C0012001393
:1004D000002F00300028004D0039000400160007EE
:1004E0000009000A000B000D000E000F003300345D
:1004F00000310000000000E100C35C1D001B00068D
:10050000001900050011001000360037003800E522
:100510000052000000E000E300E2000000000000E4
:10052000002C000000E6000000E400500051004FE5
:10053000004C00005C01000100010001000100010D
:1005400000010001000100010001000100010001A3
:100550000001000100010001000100010001000193
:100560000001000100010001000100010001000183
:100570000001000100010001000100010001000173
:100580000001000100010001000100010001000163
:100590000001000100010001000100010001000153
:1005A0000001000100010000000000010001000145
:1005B0000001000100010001000100010001000133
:1005C0000001000100C35C00000100010001000007
:1005D000000000000001000000010000000100C058
:1005E0005CC25CBE5C010001000100010001000171
:1005F00000010001000100010001000100010001F3
:1006000000010001000100010001000100010001E2
:1006100000010001000100010001000100010001D2
:1006200000010001000100010001000100010001C2
:1006300000010001000100010001000100010001B2
:1006400000010001000100010001000100010001A2
:100650000001000100010001000100000000000194
:100660000001000100010001000100010001000182
:100670000001000100010001000100000001000173
:100680000001000000000000000100000001000067
:1006900000010001000100010001001E0F0500041F
:1006A0007F3F1F643214643214783C1E1E140A0506
:1006B00009025B00030100A0FA0904000001030124
:1006C00001000921110100012240000705810308F2
:1006D000000A0904010002030000000921110100C1
:1006E00001222200070582032000010705030320E1
:1006F00000010904020001030000000921110100AA
:100700000122BC000705840320000A120110010029
:10071000000008544D0520010001020301040330CC
:100720000000000803450037003500000006034DB7
:100730000054000000040309040011241FBECFEF81
:10074000DAE0DEBFCDBF04B603FE27C08091A90466
:100750009091AA04A091AB04B091AC048730904B67
:10076000A740B04BD1F41092A9041092AA041092A1
:10077000AB041092AC0414BE84B7877F84BF0FB65D
:10078000F894A89580916000886180936000109231
:1007900060000FBEE0E0F8E3099524E0AEE9B1E0C7
:1007A00001C01D92A93AB207E1F711E0A0E0B1E063
:1007B000EAE9F5E502C005900D92AE39B107D9F727
:1007C0000E94F3220C94802A0C940000E8EDF0E0E3
:1007D00080818E7F80831092E2001092DA00109266
:1007E000E100A0EEB0E08C9181608C9380818F77E6
:1007F000808319BCA7EDB0E08C918E7F8C938081B3
:100800008F7E80831092730408952091E4003091CC
:10081000E50095E6A9012091EC00822F817020FF70
:1008200006C08091E80080FF06C080E00895209116
:10083000E80022FD1AC080919804882389F0853051
:1008400089F08091EB0085FD0FC02091E40030918C
:10085000E50042175307F9F29150E1F684E008955C
:1008600082E0089583E0089581E00895EF92FF9279
:100870000F931F93CF937C018B010E940504C82F17
:10088000811117C08091E80085FD0BC08091E800C0
:100890008E778093E8000E940504882399F3C82F7F
:1008A00008C0F70181917F018093F1000150110987
:1008B00049F78C2FCF911F910F91FF90EF900895E2
:1008C00080919A0487FF13C08091E80082FF06C0E0
:1008D0008091E8008B778093E80004C080919804B1
:1008E0008111F2CF0895809198048823D9F38091E3
:1008F000E80080FFF8CF8091E8008E77ECCF982F4A
:100900009093E900242F762F50E0891731F07091F1
:10091000EC002091ED005091F00021FD07C09F5F99
:10092000973071F78093E90081E008953091EB00F2
:100930003E7F3093EB003091ED003D7F3093ED0032
:100940003091EB0031603093EB007093EC0020931A
:10095000ED005093F0002091EE0027FDE0CF80E005
:100960000895CF92DF92EF92FF920F931F93CF9350
:10097000DF93C8EDD0E088818F7E8883E7EDF0E0DB
:1009800080818160808384E082BF81E080937304F2
:1009900088818E7F888302EE10E0F8011082109229
:1009A000DA0081EEC82ED12CF601108288818F7773
:1009B000888388818068888388818F7D888319BC3B
:1009C0001092980410929904109297041092960431
:1009D00090EEE92EF12CF70180818B7F8083888156
:1009E0008160888342E060E080E00E947F04F6013D
:1009F00080818E7F8083F801808181608083808107
:100A000088608083F70180818E7F80838881806108
:100A10008883DF91CF911F910F91FF90EF90DF902E
:100A2000CF900895FC018091A0049091A1048617B5
:100A30009707A0F06115710529F49091E8009E7761
:100A40009093E80090E06115710551F4911108C090
:100A50008091E80082FF34C080E00895BC01F2CFAD
:100A6000809198048823C1F18530C1F18091E8001C
:100A700083FD30C08091E80082FDEACF8091E800DC
:100A800080FFE1CF8091F3002091F200382F6115B3
:100A9000710519F02830310558F091E02830310502
:100AA00009F090E02091E8002E772093E800CBCF6A
:100AB00081918093F100615071092F5F3F4FE7CF23
:100AC00080919804882341F0853041F08091E800BE
:100AD00083FFBECF81E0089582E0089583E008950A
:100AE000089580E008958091750408959C014FB7A2
:100AF000F89480916F0490917004A0917104B0916A
:100B000072044FBF821B930B08952FB7F894809106
:100B10006F0490917004A0917104B09172042FBF82
:100B200008958091240481111092240408958091E5
:100B3000230490912204892B90912104892B809386
:100B4000A001909124049923A1F0892B8093A00106
:100B500080911C01882341F18091350487FF24C0D6
:100B60008EE1E2EAF1E090E0815000F591110E94FF
:100B70009105E0913804F09139043097E1F08091CB
:100B80001C01882359F08091350487FF07C08091AC
:100B9000A0018093A10185E08093A0010280F381F0
:100BA000E02D80EA91E0099486E0DBCF21912223B9
:100BB000D9F29F5FD9CF089590911C019923D1F06C
:100BC0009091350497FF16C0E82FE695E695E695D7
:100BD000EE31E0F4F0E0E056FE4F282F277081E080
:100BE00090E001C0880F2A95EAF7809592818923C9
:100BF00082830895E2EAF1E09191891303C0DF0155
:100C000011971C9291E0E83AF907B1F70895909195
:100C10001C019923C1F09091350497FF14C0E82F6F
:100C2000E695E695E695EE31F8F4F0E0E056FE4FF5
:100C3000877021E030E001C0220F8A95EAF78281B7
:100C4000822B82830895A2EAB1E0EFEF90E02D912C
:100C5000821751F0EF3F19F4211101C0E92F9F5F76
:100C60009630A9F7EF3F09F408950E2E000CFF0B04
:100C7000E056FE4FE6CF2FE0929F800D1124982F73
:100C8000977086958695869525E0829FF0011124C0
:100C9000EC51FC4F50E040E080E0219130E0092E23
:100CA00002C0369527950A94E2F721703327042E67
:100CB00001C0220F0A94EAF7822B4F5F5F4F453045
:100CC000510559F708952FE0929F800D1124982F18
:100CD000977041E001C0440F9A95EAF78695869592
:100CE000869595E0899FF0011124EC51FC4F90E02E
:100CF00080E070E05191DF0111979B01082E02C046
:100D0000369527950A94E2F721702195252724230B
:100D100025272C9301968530910561F708958091E0
:100D2000E3039091B203981301C008958F5F877019
:100D3000FACF882341F080959091230489238093F2
:100D400023040C9497050895882339F09091230487
:100D5000982B909323040C94970508952091A80351
:100D60003091A9032817390771F09093A903809354
:100D7000A803E0913804F0913904309721F0008401
:100D8000F185E02D099408952091A6033091A703E1
:100D90002817390771F09093A7038093A603E09179
:100DA0003804F0913904309721F00680F781E02D66
:100DB00009940895E0913804F0913904309721F0B6
:100DC0000190F081E02D099480E00895CF92DF92A8
:100DD000EF92FF92843030F5811125C09091800010
:100DE0009F7D909380002E98282F30E0AFEFBFEFCB
:100DF0000E94712A23E030E040E050E00E944F2A38
:100E0000C9012C3764E13607A0F469E070E00E9464
:100E1000282970938B0060938A00FF90EF90DF90F9
:100E2000CF90089583E0909180009062909380002D
:100E3000DBCF2A50374D4F4F5F4F942F832F722FA8
:100E4000662725EF38E241E050E00E944F2A690111
:100E50007A01CA01B9010E94FE289B01AC01C701B9
:100E6000B6010E94FE28672F782F892F99276115D8
:100E7000710521E08207910561F66FEF7FEFC9CF21
:100E8000282F220F220F220F90915B049770922B34
:100E900090935B04987F21E009F420E090915B043B
:100EA00020FB90F990935B040C94E606FA01811103
:100EB00001C0FB01099480915E04982F9E7F61F42C
:100EC0008170826080935E0480916104823418F0A6
:100ED00081E48093610408958635B0F38170846560
:100EE000F1CFAF92BF92DF92EF92FF920F931F93D9
:100EF000CF93DF93182F062FE901423408F041E425
:100F0000E42FF0E0E658FD4F011110C0E4915E2F90
:100F10004E2F4983E8835A83DF91CF911F910F9120
:100F2000FF90EF90DF90BF90AF900895202F30E0BA
:100F30004491D42EE42EF12C56E0159FC0011124CB
:100F4000EFEFF0E0BF010E942829812F90E0880F89
:100F5000991F55E5569FD001579FB00D11248A1B4C
:100F60009B0B982F990F890F5F01A21AB30AAE9CB1
:100F7000D001AF9CB00DBE9CB00D11245B2F089F1B
:100F800080011124012F11275F01A01AB10AAE9C24
:100F90008001AF9C100DBE9C100D11245F01A81A9A
:100FA000B108A29EC001A39E900DB29E900D112487
:100FB000892F9927E81BF90BEE9DC001EF9D900D3D
:100FC000FE9D900D1124E92F62307105A1F050F4BF
:100FD0006115710509F49DCF6130710581F0EB2F2A
:100FE000512F97CF6430710569F080F0663071053C
:100FF00009F48FCFF4CFE42F4B2F592F8ACFE42F52
:10100000412F87CFEB2F542F492F83CF4B2F5D2DAF
:10101000E12F7FCF0E9485059C019091490480912A
:101020004A04982B21F03093460420934504909174
:101030004B0480914C04982B21F03093430420936F
:101040004204E0913804F0913904309749F082E08D
:10105000809347040480F581E02D87E494E00994AF
:10106000089590E080E00E94C40690E080E00E9435
:10107000AE0610922204109221040E94970586E089
:10108000E7E4F4E0DF011D928A95E9F71092440449
:10109000109241041092AB030C940A086093A504CB
:1010A0007093A6048093A7049093A8040C9431082D
:1010B0000F931F936091A5047091A6048091A704DB
:1010C0009091A8048B019C010670112722273327D9
:1010D000063011052105310529F468601F910F9133
:1010E0000C944E08677FFACF0F931F9341E050E0B6
:1010F00060E070E004C0440F551F661F771F8A959B
:10110000D2F7CB01BA0160957095809590950091CA
:10111000A5041091A6042091A7043091A80460238F
:101120007123822393231F910F910C944E08909169
:1011300020048095892380932004282F277071F440
:10114000282F082E000C330B9217130639F08595C3
:10115000859585950E9474081092200408950F9338
:101160001F9341E050E060E070E004C0440F551F61
:10117000661F771F8A95D2F78091A5049091A604E7
:10118000A091A704B091A8048A019B01082B192BF8
:101190002A2B3B2BC901B8011F910F910C944E08CB
:1011A0006093250470932604809327049093280469
:1011B0000C94310890914904803F59F480914A047D
:1011C00087FF0DC010924A0491110BC01092440485
:1011D00008C0813F81F480914A0418169CF399233A
:1011E00081F080914B0490914C04892B09F064C0EC
:1011F000109241040895823F49F497FFF0CF109276
:10120000490480914A048111ECCFE0CF833F19F467
:101210001916ACF3E4CF20914B04893F29F4121640
:10122000F4F610924B04DBCF8A3F19F427FFD7CF97
:10123000F8CF20914C048B3F29F427FFD0CF109298
:101240004C04CDCF8C3F19F41216CCF3C8CF843F99
:1012500031F4809148048E7F80934804C0CF853F4D
:1012600021F4809148048D7FF7CF863F21F480914F
:1012700048048B7FF1CF873F21F480914804877F1A
:10128000EBCF883F21F4809148048F7EE5CF8D3FDE
:1012900031F48091AB038E7F8093AB03A0CF8E3F60
:1012A00021F48091AB038D7FF7CF8F3F09F097CF6B
:1012B0008091AB038B7FF0CF0895882309F459C048
:1012C000823871F40E94DA0681FF53C089E30E94DC
:1012D00007060E94970589E30E94DC050C94970598
:1012E000833859F40E94DA0680FF43C083E50E94E8
:1012F00007060E94970583E5EFCF843859F40E94D2
:10130000DA0682FF36C087E40E9407060E9497052E
:1013100087E4E2CF9CEF980F913AF0F290E2980FB9
:10132000983088F4877021E030E0A90102C0440FB2
:10133000551F8A95E2F7CA0180959091230489236D
:1013400080932304CBCF9BE5980F933020F490E05B
:1013500080E00C94C40698E5980F973120F490E053
:1013600080E00C94AE06803F20F00E94DA080C94D6
:101370000A0808958091AB0380FD16C081FD16C058
:1013800082FD16C0809141048823A1F0883280F448
:1013900028E0829FC001112468E270E00E943C298D
:1013A000862F672B39F0089582E0089584E0089530
:1013B00088E0089581E008958091AB0380FD14C01A
:1013C00081FD14C082FD16C080914404882381F001
:1013D000843180F422E3829FC001112464E170E033
:1013E0000E943C29862F08958CE0089589E1089594
:1013F00085E0089582E30895803F31F40E94DC097E
:10140000819580934A040895813F19F40E94DC0974
:10141000F8CF823F31F40E94DC0981958093490422
:101420000895833F19F40E94DC09F8CF893F29F41D
:101430000E94BA0980934B0408958A3F21F40E94C8
:10144000BA098195F7CF8B3F31F40E94BA09819593
:1014500080934C0408958C3F19F40E94BA09F8CF88
:10146000843F31F48091480481608093480408955A
:10147000853F21F4809148048260F7CF863F21F4B4
:10148000809148048460F1CF873F21F48091480423
:101490008860EBCF883F21F4809148048061E5CFDC
:1014A0008D3F31F48091AB0381608093AB0308954D
:1014B0008E3F21F48091AB038260F7CF8F3FB9F765
:1014C0008091AB038460F1CFF894E82FE295EF7040
:1014D000F0E031A1282F2F7081E090E001C0880F4B
:1014E0002A95EAF7982F9095932391A392A1892B9F
:1014F00082A3789408959091350492FF06C0282F16
:1015000028712830F9F4877F846093FF06C0282F64
:1015100028712831F1F4877E84612091360420FF00
:1015200006C0382F38713830D9F4877F816021FFA9
:1015300006C0282F28712831D1F4877E816194FD5F
:10154000877E0895282F24712430F9F68B7F8860D8
:10155000DCCF282F2471243101F78B7E8861DDCF09
:10156000382F3171313019F78E7F8860E0CF282F06
:101570002171213121F78E7E8861E1CFCF9384E004
:1015800090E00E94D529C82F81E290E00E94D529E1
:10159000982F8C2FCF9108950F931F93CF93DF93A4
:1015A000843030F5663020F54F3010F5C42FD0E090
:1015B000CC0FDD1F2EE1629FC00DD11D112434EB35
:1015C000839FC00DD11D1124CE0186960E94D5297E
:1015D000082F10E0102F0027CE0187960E94D529F2
:1015E0009801282BC901DF91CF911F910F91089588
:1015F00090E080E0F8CF462F843038F4763028F43D
:101600006F3018F4672F0C94CC0A90E080E00895B6
:10161000CF93DF930E94FB0AEC0182389105A9F178
:10162000D8F58133910509F496C048F589329105C2
:1016300009F48AC08A9709F495C0C11521E5D2073B
:1016400008F0BCC0C11530E5D30708F014C1C83E8E
:10165000D10508F09CC0C03ED10560F5C83AD1055F
:1016600008F087C0C53AD10508F0FDC0C130D105EA
:1016700009F12097F9F0C430D105E0F440C085337A
:10168000910509F45AC0C997C1F680913504837059
:1016900089F0C0EED0E00EC0833E910599F170F460
:1016A000803E910501F1823E910539F68091350425
:1016B00082FD21C0CE01DF91CF910895863E910534
:1016C00061F1873E910571F1843E910509F0B5CF36
:1016D0008091360481FFEECF80913504C7EED0E0D3
:1016E00084FD0DC0E7CF8091350480FD12C190913B
:1016F000360490FFDFCFC3EED0E084FFDBCFD0E035
:10170000C0E0D8CF8091350482FD06C190913604A7
:1017100090FDBFCF84FFCECFF2CF8091350483FD03
:10172000DDCFC8CF8091350483FDF9C09091360498
:1017300091FFF0CFC4EED0E0BDCF8091350485FF9E
:10174000B9CFC9E2D0E0B6CF8091350485FFB2CFE2
:10175000C5E3D0E0AFCF8091350486FFABCFCAE2BE
:10176000D0E0A8CF8091350486FFA4CFC1E3D0E0BC
:10177000A1CFCF3BD10518F6C85AD0E0CC0FDD1F62
:10178000C55BDE4F0990D881C02DD46493CFC115BD
:1017900040E2D40758F4C11581E0D80708F08ACF99
:1017A000C03FD10508F4ABCFD06584CFC11590E41C
:1017B000D90708F4A4CFDF70D06A7CCFC11525E526
:1017C000D20700F5C11534E5D30708F08AC0C1156A
:1017D00043E5D40708F071C0C11582E5D80708F4C5
:1017E00067C0CE018370992721E030E002C0220F4C
:1017F000331F8A95E2F7C695C69580E2C89FE0013F
:10180000112452C0C11599E5D907A8F4C11528E5DE
:10181000D20708F06BC0C11536E5D30708F06FCFCB
:101820008C2F0E947B0AC82FD0E0DC2FCC27CC273E
:10183000DF71D0623FCFC1154AE5D40708F45BC021
:10184000CE0190568115904208F059CF8D2F8F719F
:101850000E947B0A90E0982F882788279F719C011F
:101860002C2BE901E6CFC55AD0E0C85BDE4FC8811A
:10187000D0E0D0641FCFCE01E4E096958795EA953D
:10188000E1F783702C2F26952695237040E2249F44
:1018900090011124382B8C2F8370C1E0D0E002C05E
:1018A000CC0FDD1F8A95E2F7C22BD32BDC6802CF69
:1018B000DC2FCC27C16FD06AFDCECE018370992773
:1018C00021E030E002C0220F331F8A95E2F7C6956F
:1018D000C69590E2C99FE0011124C22BD32BDA6890
:1018E000E9CEDC2FCC27C46FD06AE4CEDC2FCC2726
:1018F000C06FD06ADFCE8C2F8F700E947B0A34E0DD
:10190000D695C7953A95E1F7CF709C2FEC01D06939
:10191000D1CEC9E3D0E0CECEC2EED0E0CBCEC6EE83
:10192000D0E0C8CEBF92CF92DF92EF92FF920F939A
:101930001F93CF93DF938C01C090A504D090A60491
:10194000E090A704F090A8048091250490912604CB
:10195000A0912704B0912804C82AD92AEA2AFB2A90
:10196000CFE1D0E0BC2ED701C6010C2E04C0B69545
:10197000A795979587950A94D2F780FD0EC0219779
:1019800088F7B12C8B2DDF91CF911F910F91FF9094
:10199000EF90DF90CF90BF900895B8018C2F0E94F8
:1019A000080B019761F3EECFCF93DF93EC010E9418
:1019B000920CBE01DF91CF910C94080B0E94D40CC5
:1019C000292F2F7092959F7092509E3078F4E92FB6
:1019D000F0E0EE57F54D0C945029803F19F020F4BB
:1019E000883E20F481E00895843FE1F380E008958B
:1019F000883EC0F3813FD1F7F5CF822F869586953B
:101A000086950895682F86E090E00C94E929CF939D
:101A1000DF93C6EFD2E060E0CE010E94E929219673
:101A2000C11584E0D807B9F7DF91CF9108951F93CE
:101A3000CF93DF93122F8430F8F46630E8F44F3000
:101A4000D8F4C42FD0E0CC0FDD1F9EE1699FC00DFC
:101A5000D11D112494EB899FC00DD11D1124632F3A
:101A6000CE0186960E94E929612FCE018796DF91EB
:101A7000CF911F910C94E929DF91CF911F91089587
:101A8000AF92BF92CF92DF92EF92FF921F93CF93CC
:101A9000DF938FE7C82E84E0D82ED0E07601C0E037
:101AA00014C0F50125913491412F6C2F8D2F0E9488
:101AB000170D82E0A80EB11C1F5F1F3091F78EE159
:101AC000E80EF11CCF5FC63019F0570110E0E9CFE6
:101AD000DF5F84EBC80ED11CD43001F7DF91CF91CA
:101AE0001F91FF90EF90DF90CF90BF90AF9008953F
:101AF000CF93DF9300D00F92CDB7DEB790919804CB
:101B0000943011F589837B836A839093E9008FEF8A
:101B10009091E800815095FD06C095ED9A95F1F7FA
:101B200000008111F5CF8091E80085FF0DC050E0E5
:101B300040E063E070E0CE0101960E94360480919F
:101B4000E8008E778093E8000F900F900F90DF9160
:101B5000CF910895BC0184E00C94780DBC0183E022
:101B60000C94780D9C0184E08093E9009FEF8091B4
:101B7000E800915085FD06C085ED8A95F1F70000DB
:101B80009111F5CF8091E80085FF0CC050E040E056
:101B900066E070E0C9010E9436048091E8008E770B
:101BA0008093E8000895CF93DF93EC0180911C01AE
:101BB0008823B1F18091350487FF32C060E284E070
:101BC0008093E9008FEF9091E800815095FD06C069
:101BD00095ED9A95F1F700008111F5CF8091E8001D
:101BE00085FF1BC080911C0170E050E040E0811136
:101BF00004C050E040E068E070E0CE010E9436048E
:101C00008091E8008E778093E80080E2FE01A6E7ED
:101C1000B4E001900D928A95E1F7DF91CF9108959C
:101C200068E081E0CDCF81E08093E00080E28093A6
:101C3000D8001092C9008FE19EE40197F1F700C02F
:101C4000000087E090EBDC018093A9049093AA0444
:101C5000A093AB04B093AC0488E19CE00FB6F89479
:101C6000A895809360000FBE90936000FFCFCF9344
:101C7000C82F882309F4AEC08238C1F40E94DA0666
:101C800081FDA8C089E30E9407060E9497052FEFF7
:101C900081EE94E0215080409040E1F700C00000C8
:101CA00089E30E94DC05CF910C9497058338A1F459
:101CB0000E94DA0680FD8EC083E50E9407060E941E
:101CC00097052FEF81EE94E0215080409040E1F79E
:101CD00000C0000083E5E5CF8438A1F40E94DA0655
:101CE00082FD78C087E40E9407060E9497052FEFC7
:101CF00081EE94E0215080409040E1F700C0000068
:101D000087E4CFCF8CEF8C0F813A88F580911C014E
:101D1000882301F18091350487FF1CC0EC2FE695E4
:101D2000E695E695F0E0E056FE4F828190E04C2F7C
:101D3000477021E030E002C0220F331F4A95E2F7DE
:101D400082239323892B79F08C2F0E94DC050E943B
:101D5000970509C0E2EAF1E08191C817A9F321E0F3
:101D6000E83AF207C9F78C2F0E9407069CCF80E261
:101D70008C0F883068F4C77021E030E001C0220F7A
:101D8000CA95EAF780912304822B809323048BCF9A
:101D9000EBE5EC0FE33040F4F0E0E85BFE4F8081D0
:101DA00090E0CF910C94C406E8E5EC0FE73150F4D5
:101DB000F0E0EE0FFF1FE55BFE4F80819181CF9138
:101DC0000C94AE06C03F30F08C2F0E94FC09CF91DE
:101DD0000C940A08CF9108951F93CF93DF93182F87
:101DE000D0E0C0E0893311F4C0E5D0E0812F0E943B
:101DF000370E209731F4812FDF91CF911F910C94F2
:101E00005D098FE99FE00197F1F700C0000021977D
:101E1000F0CF0F931F93CF93DF93C62FD42F022FB2
:101E2000FC0182818823A1F06093A4040E948505AF
:101E30009093A3048093A204C77081E001C0880F2F
:101E4000CA95EAF7DF91CF911F910F910C94A406E8
:101E50008091A404681335C08091A2049091A304DA
:101E60000E947605883C910560F510E21D0FCD17A4
:101E7000B9F080E28C0F883040F4C77081E001C077
:101E8000880FCA95EAF70E949906183048F481E055
:101E90009D2F977001C0880F9A95EAF70E94A406BB
:101EA000802F0E94EC0E183098F4D77081E001C0AA
:101EB000880FDA95EAF7DF91CF911F910F910C947B
:101EC0009906C77081E001C0880FCA95EAF7F3CF81
:101ED000DF91CF911F910F91089580915E0480FD55
:101EE0000AC0E6ECF1E0118210821282339652E0D1
:101EF000EA37F507C1F76A9A3EB13B7F2EB12460FD
:101F00004FB7F89486EC91E0FC015191CF0168E065
:101F10002EB9000000C057FF3EB9550F000000C0A9
:101F200000C000C03EB900C06A9591F7F2E08A3760
:101F30009F0751F74FBF8FE594E00197F1F700C07D
:101F400000000895EF92FF921F93CF93DF93EC016F
:101F500086ECE82E81E0F82E10E08C81970140910C
:101F6000610460916004810F0E9471071C5F83E02F
:101F7000E80EF11C103F89F70E946D0F9A818C8149
:101F800090FF08C08F5F8C83DF91CF911F91FF90EE
:101F9000EF9008958150F7CFBF92CF92DF92EF92EA
:101FA000FF920F931F93CF93DF93FC018281DD2477
:101FB000DA9480FD02C0DD24D39406EC11E0D0E079
:101FC000C0E02CE3B22EF80111821082128294E05C
:101FD000E92EF12CC12C8091C3018C0D8D330CF4B2
:101FE0003DC06B2D0E941A29892F082E000C990BD9
:101FF0008C179D0791F4809161048E9DA0018F9DA7
:10200000500D112455954795559547959801609128
:10201000600480915F040E947107CD0CF1E0EF1A1B
:10202000F108C9F621960D5F1F4FCC33D10559F643
:102030000E946D0F8091C30191E0D91215C08111EA
:1020400011C08BE38093C301DF91CF911F910F915A
:10205000FF90EF90DF90CF90BF90089587FFC5CF9E
:10206000845CC3CF8150EECF90E00196BE010E9408
:102070003C29E8CF0F931F93CF93DF93C6ECD1E0B9
:10208000FE01118210821282339682E0EA37F8074D
:10209000C1F710E000E08091C401082E000C990BFC
:1020A000081719078CF180911001082E000C990B6C
:1020B000801791074CF19E0140916104609160048A
:1020C00080915F040E9471070F5F1F4F23960C33AE
:1020D000110509F70E946D0F80910F019091C401C5
:1020E000980F9093C40120911001280F20931001A4
:1020F000121614F49B331CF0819580930F01DF912D
:10210000CF911F910F910895198218821A82DCCF06
:102110008F929F92AF92BF92CF92DF92EF92FF92F7
:102120000F931F93CF93DF93EC014C81042F10E0AA
:102130009801D8010E94712A9B01AC010E943C2A9F
:102140004B015C01E0E2F0E0E01BF10BA5E5B0E043
:10215000AC019B010E943C2A6B017C019F01DF01C5
:102160000E945D299B01AC010E94472A9B01AC01A2
:10217000280D391D4A1D5B1DC701B6010E944F2A5B
:10218000F22E822F90E039E23F15D8F143E0249FF0
:102190009001112435952795122F109596ECC92E94
:1021A00091E0D92E00E085E5E82EEF188E2D01FD97
:1021B0008F2D9601412F609160040E9471070F5F7F
:1021C00053E0C50ED11C0C3389F70E946D0F9C8122
:1021D00081E0992319F0903219F48FEF8093110167
:1021E00080911101890F8C83DF91CF911F910F9105
:1021F000FF90EF90DF90CF90BF90AF909F908F9027
:10220000089525E530E0A901481B590BCA019A0140
:10221000220F331F280F391F37FFBCCF2F5F3F4FCF
:10222000B9CFEF92FF920F931F93CF93DF938C015F
:10223000C6ECD1E0F12CE12CF801948160916004AE
:1022400080915F04FEE1EF16F104FCF49923F9F0AC
:102250009E01409161040E9471072FEFE21AF20A79
:1022600023968CE3E816F10439F70E946D0FF8010C
:10227000848190E00196817099278483DF91CF91CA
:102280001F910F91FF90EF900895992309F39E01FC
:1022900040E0E1CF90915E0490FF0CC0E6ECF1E0ED
:1022A000818360834283339692E0EA37F907C1F76E
:1022B0000C946D0F08950F931F93CF93DF9300D06D
:1022C0000F92CDB7DEB78C018091C50181110AC094
:1022D0009E012F5F3F4F41E46FEF0E9471078A819B
:1022E0008093C501F8016481613069F08091C50176
:1022F00040E0662361F040E0623011F44091C50196
:1023000080E060E004C06091C50140E080E00E9490
:102310004A11F801848190E0019663E070E00E9428
:102320003C2984830F900F900F90DF91CF911F91E4
:102330000F910895CF93DF9300D00F92CDB7DEB702
:1023400090915E0490FF0AC09E012F5F3F4F0E9454
:1023500071074B8169818A810E944A110F900F9009
:102360000F90DF91CF910895CF93DF93EC01EC8133
:10237000F0E0E158FC4F4491EEE5F4E062818181A8
:102380000E949A118C818F5F8C83DF91CF91089589
:10239000CF93DF93EC01EEE5F4E0438162818C8121
:1023A0000E949A118C818F5F8C83DF91CF91089569
:1023B0006F927F929F92AF92BF92CF92DF92EF92F5
:1023C000FF920F931F93CF93DF9399E7E92E91E04C
:1023D000F92ED0E0C0E010E0CC24C394D12C35E33A
:1023E000A32E34E0B32ED7018D917D01F894E82F10
:1023F000E295EF70F0E021A18F70A60102C0440FBA
:10240000551F8A95E2F7CA01922F982B91A392A1AA
:102410008095892382A3789400C0A6010C2E02C067
:10242000440F551F0A94E2F7BA0160957095E9E2EE
:10243000F4E088E8682E81E0782E00E02191319167
:10244000D3019D903D01892D82958F7090E0DC0134
:1024500090968C9190E0B92DBF7002C095958795AC
:10246000BA95E2F780FD67C0C901842B952B281728
:10247000390739F09F0122503109D9018D939C937E
:1024800001E0AE16BF06D1F6F701319780810E94B8
:10249000640ACE3019F0E0EAEA95F1F7102B2196A4
:1024A000CF30D10509F09FCF112309F448C081E056
:1024B0008093C2010E9485059093C1018093C00161
:1024C0008091C0019091C1010E9476050697D8F1D4
:1024D0008091290490912A0490936404809363046A
:1024E00080912B0490912C04909366048093650452
:1024F00080912D0490912E0490936804809367043A
:1025000080912F049091300490936A048093690421
:10251000809131049091320490936C0480936B0409
:10252000809133049091340490936E0480936D04F1
:102530001092C20108C0C9018623972398CF8091C9
:10254000C2018111BDCF812FDF91CF911F910F91DA
:10255000FF90EF90DF90CF90BF90AF909F907F90D3
:102560006F900895AF92BF92CF92DF92EF92FF9259
:102570000F931F93CF93DF93EC018AE0A82E28815D
:10258000222309F48CC02130C9F599818A819130C8
:1025900021F422960E94EC0E05C0923029F4229676
:1025A0000E94370E2196EBCF933021F422960E94A1
:1025B0005D09F8CF943011F02196F4CF229630E0E7
:1025C00020E0AE014F5F5F4F8053990B8A30910539
:1025D00050F02150310930F38FE99FE00197F1F776
:1025E00000C00000F6CFA29EB001A39E700D112482
:1025F0009C01260F371F8981EA01E3CFE22FF0E02B
:10260000E650FE4FB490822F86958695869590E091
:10261000FC01E651FE4FE4902770F12C022E02C01F
:10262000F594E7940A94E2F731E0E322FF24FC01F9
:10263000E652FE4FC490D12C022E02C0D594C7940E
:102640000A94E2F731E0C322DD24FC01E653FE4F99
:10265000049110E002C0159507952A95E2F70170E4
:102660001127E114F10419F081EE0E94370EC11414
:10267000D10419F086EE0E94370E8B2D0E94EC0ECD
:10268000CD2819F086EE0E945D09EF2819F081EE41
:102690000E945D09012B09F485CF8CE27BCFDF918D
:1026A000CF911F910F91FF90EF90DF90CF90BF904F
:1026B000AF9008954F925F926F927F928F929F9208
:1026C000AF92BF92CF92DF92EF92FF920F931F9340
:1026D000CF93DF93FC016280448081E08483EFE745
:1026E000F3E07490EEEFF3E0E491CAE7D2E036EC69
:1026F000E32E31E0F32E46EAC42E43E0D42E52E01E
:10270000A52EBB24B39488248A94912C55245A94E2
:10271000E7190E2F10E082E0861530F080915F04FB
:102720008883809160048983411021C01B821A82B2
:1027300097014A81698188810E947107259683E00B
:10274000E80EF11CCC16DD0631F7DF91CF911F9119
:102750000F91FF90EF90DF90CF90BF90AF909F9040
:102760008F907F906F905F904F900C946D0F8B8146
:102770008823E9F081508B83859DC00111246C81F1
:1027800070E00E942829FB01FF27E158FC4F84914B
:10279000E82FE719E59DC0011124B8010E942829FE
:1027A00080916104689FB00111247A83C1CF0E9497
:1027B000B82920916104269521582A9DA0012B9DBE
:1027C000500D1124452F5527841795070CF0B0CFD5
:1027D00082E0861588F40E94B829B4010E943C2941
:1027E00088830E94B829209160042695622F70E0AA
:1027F0000E943C29280F29831A8280916104893C18
:1028000020F088EC8C838B8393CF8431D8F784E1DC
:10281000F9CF90E080E00E94E32921E08B3E9E4FBB
:1028200009F020E0822F08956BEE7EEF90E080E0CB
:102830000E94072A60E082E090E00E94E92960E0BF
:1028400083E090E00E94E92910922504109226046A
:10285000109227041092280460E084E090E00E9427
:10286000E92960E081E290E00E94E92960E085E0EA
:1028700090E00E94E92960E086E090E00E94E9296A
:102880006FEF87E090E00E94E92940E050E0BA0154
:1028900088E090E00E94FB2960E08DE090E00E94DB
:1028A000E92940E050E0BA0188E190E00E94FB296C
:1028B00060E087E190E00E94E92940E050E0BA0141
:1028C0008CE190E00E94FB2960E080E290E00E94B1
:1028D000E92940E050E0BA0188E190E00E94FB293C
:1028E00040E050E0BA018FE090E00E94FB2940E018
:1028F00050E0BA0183E190E00C94FB290E94091496
:10290000811102C00E94141486E090E00E94D52933
:1029100080935B04803220F08770886180935B0431
:1029200090915B04892F817090FF04C0892F869558
:10293000869586950C94E606CF92DF92EF92FF92F1
:102940006B017C010E945B07B701A60188E090E063
:10295000FF90EF90DF90CF900C94FB295F926F92E5
:102960007F928F929F92AF92BF92CF92DF92EF921F
:10297000FF920F931F93CF93DF9300D00F92CDB7A9
:10298000DEB7182F762E042F622E90915E0490FFF2
:1029900029C0E92FE695AE2FB0E0A35EBE4F8C9123
:1029A00080935C049E7F923081F59E012F5F3F4FA4
:1029B000812F0E9471074B8169818A810E944A118F
:1029C00010935F047092600400936104662051F0DC
:1029D00060915E0470915F04809160049091610445
:1029E0000E949C140F900F900F90DF91CF911F9138
:1029F0000F91FF90EF90DF90CF90BF90AF909F909E
:102A00008F907F906F905F900895823019F40091BD
:102A10006104D6CF863019F410915F04D1CF89308C
:102A2000D9F3893169F6E9518E2F8170582EE695D8
:102A3000F0E0E658FC4FA590B490BB2486ECE82E5D
:102A400081E0F82ED12CC12C9CE3892E912CC6015B
:102A5000B4010E942829812F511013C0860F9701BD
:102A6000402F672D0E947107CA0CDB1C83E0E80E23
:102A7000F11C8AE7E81682E0F80649F70E946D0F1C
:102A80009FCF861BECCFEEE5F4E0438128E0421BAC
:102A900008F440E021E0628181810C94AE14EEE5FF
:102AA000F4E0438128E0420F08F44FEF21E0628117
:102AB00081810C94AE14EEE5F4E0628128E0621BA3
:102AC00008F460E021E0438181810C94AE14EEE5CE
:102AD000F4E0628128E0620F08F46FEF21E04381A7
:102AE00081810C94AE14EEE5F4E0818121E0438114
:102AF000628188500C94AE14EEE5F4E0818121E00F
:102B000043816281885F0C94AE14809162048823B3
:102B100019F081508093620460915E0470915F04AB
:102B200080916004909161040C949C1480916204E3
:102B3000833018F48F5F8093620460915E0470911B
:102B40005F0480916004909161040C949C14EEE504
:102B5000F4E083E0808311828FEF828381E48383BA
:102B6000148260817181828193810C949C141092F3
:102B7000230480911C01E2EAF1E0882359F080915E
:102B8000350487FF07C08EE1DF011D928A95E9F7C2
:102B90000C94310886E0F8CF1F93CF93DF93CDB725
:102BA000DEB7AA970FB6F894DEBF0FBECDBF8AE995
:102BB00094E02091F100DC012D93CD01B4E0823A44
:102BC0009B07B9F780919B04833009F471C0B8F476
:102BD000813009F448C0823009F4B2C08091E80025
:102BE00083FF3AC180919A0490919B049A3008F037
:102BF00033C1E92FF0E0E057F54D0C9450298A30AD
:102C000009F48DC08B3009F470C0893039F7809198
:102C10009A04813219F780919E0490919F04009745
:102C200011F00297D9F68091E800877F8093E80041
:102C30008091E80082FF37C09091F3008091F2000C
:102C4000029729F48091F1008B7F813021F48091EB
:102C5000F100809375048091E8008B778093E80001
:102C60000E946004BBCF80919A04813A09F0B6CFEC
:102C70008091E800877F8093E80080919E04909186
:102C80009F04892B61F460E286E794E070E00E9483
:102C900012058091E8008B778093E8009FCF60E079
:102CA00090E080E0F3CF809198048111C1CF96CF5E
:102CB00080919A04813A09F091CF80919E0490917D
:102CC0009F04892B09F08ACF8091E800877F809349
:102CD000E8008091E80080FFFCCF80911C01809388
:102CE000F1008091E8008E77B9CF80919A0481320B
:102CF00009F074CF80919E0490919F04892B09F074
:102D00006DCF8091E800877F8093E8000E94600487
:102D100080919C0480931C010E94B7155FCF809125
:102D20009A04813209F05ACF8091E800877F80931E
:102D3000E8000E94600480919D04809374044ECF4B
:102D400080919A04813A09F049CF8091E800877F09
:102D50008093E8008091E80080FFFCCF80917404AC
:102D6000BECF803899F0823809F076C080919E04F9
:102D70008F70873008F070C08093E9008091EB007D
:102D800085FB882780F91092E90006C0809196049F
:102D900090919704911182609091E800977F9093B1
:102DA000E8008093F1001092F1008091E8008E77A6
:102DB000C0C1882309F4ADC1823009F04DC08091B3
:102DC0009C048111B1C180919E048F702FEF280F58
:102DD000263008F041C08093E9002091EB0020FFED
:102DE000A3C1933031F48091EB0080628093EB00BB
:102DF0009BC19091EB0090619093EB0021E030E05B
:102E000001C0220F8A95EAF72093EA001092EA00A7
:102E10008091EB008860EACF81111EC010919C0464
:102E20001F778091E3008078812B8093E30080916D
:102E3000E800877F8093E8000E9460048091E800AA
:102E400080FFFCCF8091E30080688093E30082E004
:102E5000111183E0809398048091E80083FF0AC0F9
:102E60008091E800877F8093E8008091EB0080628A
:102E70008093EB00AA960FB6F894DEBF0FBECDBFCD
:102E8000DF91CF911F9108958058823028F72091CB
:102E90009C0430919D042C3DE3E03E07A1F583E0C6
:102EA0008A838AE289834FB7F894DE01139620E083
:102EB0003EE051E2E32FF0E050935700E49120FF11
:102EC00003C0E295EF703F5FEF708E2F90E0EA3025
:102ED000C0F0C7968D939D932F5F243159F74FBF54
:102EE0008091E800877F8093E8006AE270E0CE017D
:102EF00001960E9412058091E8008B778093E8008C
:102F0000ABCFC096E7CF80919E0490919F04432F52
:102F100055274330510509F44AC078F54130510531
:102F200009F485C08BE590E0E0EBF6E04230510516
:102F300009F092CF2091E800277F2093E8002091AC
:102F4000A0043091A1048217930708F49C0140E08B
:102F50002115310509F070C041116EC08091E80063
:102F600082FDC9CF80919804882329F2853019F217
:102F70008091E80083FFF2CFBECF4132510509F4C2
:102F800047C04232510509F067CF8330910508F000
:102F900063CFFC01EE0FFF1FEF56FE4F0190F08153
:102FA000E02D82579E4FDC018C9190E01DC03327AD
:102FB00021303105E9F02115310579F02230310554
:102FC000F9F02330310509F047CFEDE1F7E0E49166
:102FD0008E2F90E0EDE1F7E007C0E5E3F7E0E49144
:102FE0008E2F90E0E5E3F7E0009709F435CFA2CF0C
:102FF000EDE2F7E0E4918E2F90E0EDE2F7E0F4CF20
:10300000E3E2F7E0E4918E2F90E0E3E2F7E0ECCF2B
:103010008330910508F020CF880F991FFC01E956F5
:10302000FE4F0190F081E02D89E090E083CF82E1B6
:1030300090E0EBE0F7E07ECF80919804882309F4DC
:103040005ACF853009F457CF8091E80083FD53CFE4
:103050008091E80082FD82CF8091E80080FF78CFE8
:103060009091F3008091F2002115310519F088301C
:10307000910550F041E0089709F040E08091E800A8
:103080008E778093E80064CF44914093F1003196AD
:10309000215031090196E8CF803809F0DDCE8091CA
:1030A000E800877F8093E800809199048093F10085
:1030B0007CCE8111D1CE10919C04123008F0CCCE80
:1030C0008091E800877F8093E800109399040E9424
:1030D0006004112311F084E005C08091E30087FDB6
:1030E000FACF81E08093980442E061EC81E00E9495
:1030F0007F0442E261EC84E00E947F0442E261ECE2
:1031000082E00E947F0442E260EC83E00E947F0440
:10311000A3CE80919C04813009F09ECE81E0933053
:1031200009F080E0809397041092E9008091E80014
:10313000877F8093E8000E9460048ECE90915E04A9
:1031400090FF3DC09170811129C0926090935E0400
:10315000662351F060915E0470915F048091600479
:10316000909161040E949C1460915E04669570E0E9
:103170004BE050E084E091E00E94C829892BA9F03F
:1031800010925D0481E080933E0420E04091610450
:103190006091600480915F040C94AE148B3210F047
:1031A0009465D4CF880F982BD1CF81E080935D04B4
:1031B0000E94850590933C0480933B04E3CF0895DF
:1031C00080915E048695815009F48AE261E00C9456
:1031D0009E1880915E0486958F5F8B3208F081E0A7
:1031E00061E00C949E1890915E0490FF07C0969544
:1031F000981720F0961710F40C94E91861E00C94DD
:103200009E184F925F926F927F928F929F92AF9291
:10321000BF92CF92DF92EF92FF920F931F93CF93C3
:10322000DF9300D000D00F92CDB7DEB77C01FC0158
:1032300083819481892B31F08081918189238F3F13
:1032400009F0C4C50F900F900F900F900F90DF9171
:10325000CF911F910F91FF90EF90DF90CF90BF9093
:10326000AF909F908F907F906F905F904F90089558
:103270000E94920C182F682F89819A810E94630600
:1032800069817A81812F0E94FB0A8C01F70192816A
:10329000992309F470C5980122513F452031310529
:1032A00008F030C58FEF93E00E94D5294EEED42E62
:1032B000D00E06EF12E08823D1F0809120048770B1
:1032C00009F4C0CFF7018281882309F4BBCF82E0E3
:1032D0000E949708B7CF0115F4E01F0771F3C801EA
:1032E0000E94D529811101C0DA940F5F1F4FD110C0
:1032F000F2CF19821A821B821C82CC24CA94480104
:103300002FEF821A920AC8010E94D52989831A8256
:10331000882399F2813009F047C0580132E0A30EAA
:10332000B11CC4010E94D529982E8A83882329F2D2
:10333000C5010E94D529D82E8FEF890D833068F4FE
:10334000580143E0A40EB11CDB82DD2021F0CE0148
:1033500001960E94B2128501D2CF54E09512FBCFA4
:10336000580184E0A80EB11CC80103960E94D5291B
:10337000DD2009F4A2CF882309F49FCF8150990B57
:10338000C89E9001C99E300D1124ED2DE150FF0B18
:10339000CF01820F931F0197F0F2EFE9FFE0319721
:1033A000F1F700C00000F7CFCE0101960E94B212E3
:1033B0005401D1CF81E00E94AF080E9458087DCF10
:1033C00081E00E947408F9CF82E0F5CF82E0F9CF66
:1033D0000F3B8CE5180709F44AC098F1003CFCE566
:1033E0001F0709F0ABC490915B04892F86958695E1
:1033F00086958F5F8F719770843008F059C0880F61
:10340000880F880F892B80935B0480915B0410C028
:1034100083E00E94400780915B040E94020D4DCF23
:1034200080915B04982F987FE9F1885080935B042A
:10343000887F91E009F490E080915B0490FB80F933
:1034400013C080915B04982F96959695969593302E
:1034500040F49F5F990F990F990F8770892B809384
:103460005B0480915B04816080935B0419C0809150
:103470005B0480FF09C08E7F80935B040E94020D75
:1034800080E00E94E60619CF80FD17CF816080930F
:103490005B04813019F489E080935B0480915B04C4
:1034A0000E94020D80915B04869586958695E9CFF2
:1034B00090935B04AACF27E245EE65EE58C426E25E
:1034C00041EE60EE54C427E245EE64EE50C426E2BD
:1034D00041EE62EE4CC428E241E0EFCF809135042A
:1034E000806106304CE5140709F489C080913504E9
:1034F000886007301C4508F482C0809135048062E2
:103500007EC00C308CE5180709F48EC070F48091F1
:1035100035048C600A30ECE51E0709F470C008F42D
:103520007DC0809135048E7F6AC080913504877F8D
:103530000E302CE5120709F462C0809135048B7FB0
:103540000F301C4508F45BC0809135048F7E57C056
:103550000B3F4CE5140709F459C030F503318CE5F5
:10356000180709F46DC078F40131ECE51E0709F481
:1035700063C002311C4509F08BC40E94B7158091CD
:1035800035048F773CC005312CE5120709F460C083
:1035900008F474C08091360481600A3F1C4509F02C
:1035A00077C48093360474C40F3F5CE5150709F4B3
:1035B0004BC088F4809136048D7F0D3F9CE5190740
:1035C00081F3809136048E7F0E3F1C4550F380912D
:1035D00036048360E6CF0130FDE51F0709F457C0CC
:1035E00008F442C060E002301D4509F051C48EE08D
:1035F00090E00E94E9294CC4809135048160809359
:10360000350446C4809135048460F9CF8091360436
:103610008260C7CF809135048064F1CF0E94B715D6
:10362000809135048068EBCF809135048D7FE7CFA2
:10363000809135048F7DE3CF809135048F7BDFCF80
:1036400080913504837FDBCF809136048C7FA9CFB6
:103650008091350482FB992790F921E0922790FB15
:1036600082F990FB83F9CBCF80913604982F909507
:1036700091708E7F892B90FB81F993CF0E94B715B3
:1036800090913504892F97FB87F98058B8CF61E076
:10369000AECF8091230406314CE5140709F0A7C38F
:1036A0008A7A91E009F490E09093AA03811106C010
:1036B00089E20E9407060E949705FFCD85E3F9CFB6
:1036C00085E381C380915E0480FF1BC08E7F809361
:1036D0005E0460915E0470915F048091600490913B
:1036E00061040E949C1410925D045FEF80E792E0F9
:1036F000515080409040E1F700C000000E946D0FE3
:10370000DCCD816080935E0461E086950E949E1806
:10371000D4CD40EE58E169EE78E10E945607CDCD58
:1037200049EE58E160EE78E1F8CF43E755E16CE708
:1037300075E1F3CF4CE755E163E775E1EECF4BE57B
:1037400055E167E675E1E9CF47E655E16BE575E1DF
:10375000E4CF43E455E16FE475E1DFCF4FE455E199
:1037600063E475E1DACF45E855E166E975E1D5CF67
:1037700046E955E165E875E1D0CF61E081E0C6CF6B
:1037800065E082E00E94F31898CD68E086E0FACF09
:103790006EE089E0F7CF64E18FE0F4CF67E185E187
:1037A000F1CF61E088E1B2CF62E289E1EBCF61E085
:1037B00083E2ACCF0115ECE51E0709F445C00E3DD0
:1037C0001C4509F44EC0F70100811181992309F4C9
:1037D0004BC0C8010E94920CD82E682FC8010E94CD
:1037E0006306B8018D2D0E94080B8C01882EF7010D
:1037F000D280A580A2943FE0A3228091200487700C
:10380000A1F0CD2CDD2091F0812F807F803421F03C
:1038100080E2800F883048F082E00E949708809113
:1038200020048770CC24C3948111C12CB12EB29492
:103830002FE0B222FBE0FB1508F450C0EB2DF0E0C6
:10384000E656F54D0C9450290E94B7152FEF34E33E
:103850004CE0215030404040E1F700C000000E94A1
:10386000130E0E94141429CDC8010E943B06D82EC5
:10387000B8CF212F2F70A22E107F19F0A29490EFB5
:10388000A922DD20C9F0AA2069F080E2800F8830EB
:1038900010F081100BC080912304A82AA092230469
:1038A0000E949705802F0E94370E18C08091220435
:1038B000A82AA0922204F4CF802F0E945D09AA209A
:1038C00069F0A094005E083010F0811028C080914B
:1038D0002304A822A09223040E9497052B2D285090
:1038E000330B2430310510F40E94DA06CC2009F4A1
:1038F000A9CC8091200480FDA5CCF701128285958A
:10390000859585950E94AF08C7010E940119809195
:1039100020048595859585950E94740893CC8091A7
:103920002204A822A0922204D7CF312F3F70932ED9
:10393000107F103219F0929480EF9822882071F055
:1039400041E0841661F1DD20B9F1AA2071F1F7019F
:10395000858180FFA7CF8F70858327C0DD2091F000
:1039600090912404892D892BA11003C00E94A406E4
:10397000B5CF51E0A512FACF981709F4AFCF8093D5
:103980002404ACCFA11006C00E949105892D0E948D
:103990009906A4CF81E0A81609F4A0CFF5CFDD20C9
:1039A00031F095E09A1508F499CF892DDFCFE4E046
:1039B000EA1508F493CFEACFAA2041F3F9E38F1276
:1039C00009C02FEF37EE43E0215030404040E1F78F
:1039D00000C00000802F0E945D0980CF812F869556
:1039E0008695837061F0813009F078CFC8019370BB
:1039F000D11002C090E080E00E94AE066FCFC801F7
:103A00009370D11002C090E080E00E94C40666CF9F
:103A1000802FDD2039F00E94FC090E940A080E94D4
:103A20000A085CCF0E94DA08FACF812F837009F070
:103A300066C0D11053CF802F829586958770880FEE
:103A4000880F602F6F70462E512C712C612C082E20
:103A500004C0440C551C661C771C0A94D2F740E045
:103A600050E0BA0104FF0FC04FE050E060E070E0AA
:103A700004C0440F551F661F771F8A95D2F74095E3
:103A8000509560957095812F8695869583708230CC
:103A900019F1D8F4009125041091260420912704EF
:103AA00030912804813069F0442955296629772905
:103AB000CB01BA0160237123822393230E94D00893
:103AC0000DCF402A512A622A732ACB01BA016429F8
:103AD000752986299729F2CF4429552966297729FE
:103AE0000091250410912604209127043091280488
:103AF000CB01BA016027712782279327DFCF8695F4
:103B0000DD2011F0812F8170882309F4E7CE802F0A
:103B1000829586958770880F880F602F6F70462E6C
:103B2000512C712C612C082E04C0440C551C661CB1
:103B3000771C0A94D2F740E050E0BA0104FF0FC0AE
:103B40004FE050E060E070E004C0440F551F661F76
:103B5000771F8A95D2F74095509560957095812F83
:103B6000869586958370823019F1D8F40091A5046A
:103B70001091A6042091A7043091A804813069F027
:103B80004429552966297729CB01BA01602371237D
:103B9000822393230E944E08A1CE402A512A622AF2
:103BA000732ACB01BA016429752986299729F2CF96
:103BB00044295529662977290091A5041091A60466
:103BC0002091A7043091A804CB01BA016027712786
:103BD00082279327DFCF1F70DD2029F0812F0E94DD
:103BE000AF08802FC3CE802F0E949906812F0E949C
:103BF000740874CE802F52EF851609F450C0581502
:103C000078F090EF891619F1E1EF8E1609F43FC0B4
:103C1000DD2009F467C0A11045CE812F8F713CC013
:103C2000F3EF8F1609F440C024EF8212F1CFDD20AC
:103C300009F44DC01F71812F0E94AF0858E0159FF5
:103C4000C0011124836080932004812F25C0DD20D2
:103C5000C9F034E03A1508F441CE1F7161E070E01C
:103C600080E090E004C0660F771F881F991F1A95A7
:103C7000D2F70091A5041091A6042091A7043091D9
:103C8000A804A4CF45E04A1508F428CEE6CF812F3A
:103C90008F71DD2009F4ABCF0E94AF081FCE812FBA
:103CA0008F71DD20C9F3A3CF60E070E0CB01DD2090
:103CB00009F470CF1F7161E070E080E090E004C013
:103CC000660F771F881F991F1A95D2F763CF81E07F
:103CD0000E94970881E08A1508F000CE82E00E94D9
:103CE0009708FCCDAA2059F0893309F073CE9FEFD5
:103CF000E7EEF3E09150E040F040E1F769CE812F2C
:103D00008F7175CF0031FFE51F0709F453CB0131E7
:103D10002FE5120709F458CB0D3B2CE5120709F4E7
:103D20007FCB08F055CB0B3B4CE5140709F470CB67
:103D300080E00C3B5CE5150709F46BCB033F2CE5F9
:103D4000120709F4BCCB08F05EC0083D4CE514072F
:103D500009F4B1CB093D5CE5150709F4BCCB073D7F
:103D60008CE5180709F05BC026E241EE61EEC70161
:103D70000E94090FA2CA00313FE5130709F420CBC6
:103D800001314FE5140709F421CB033F3CE513074C
:103D900009F495CB08F08CC0083D5CE5150709F4E3
:103DA0008ACB093D8CE5180709F495CB073DECE576
:103DB0001E07D1F206311C4509F005CD8091AA03FA
:103DC00081117ECC89E20E94DC0575CC85E0DE01A4
:103DD000119601900D928A95E1F7F7012281898170
:103DE0009A81211145CA0E943B06182F49CA827246
:103DF000F801E25CFC45E431F10508F0DBCCEA5562
:103E0000F54D0C945029053FECE51E0709F45FCBF6
:103E100008F459CB063F2CE5120709F455C010925F
:103E2000A40402302CE5120708F433CC06313CE53B
:103E3000130738F098012A5F3C452930310508F016
:103E400028CC0E94BE0A909336048093350400313A
:103E50004CE5140709F4ECCB08F07ACB08308CE57C
:103E6000180709F4D7CB08F04CCB0430ECE51E075B
:103E700009F4C8CB08F032CB02302CE5120709F464
:103E8000BBCB80913504826003301C4509F4B7CB6D
:103E9000609135041091360484E090E00E94E92995
:103EA000612F81E290E00E94E9290E94B71505CABE
:103EB000053FFCE51F0709F40ACB08F404CB063FD5
:103EC0003CE5130709F076CF27E245EE66EE4FCFCB
:103ED0001F93CF93DF938091B103807FA9F48091EA
:103EE000AE03882389F08091E303D091B2036091FF
:103EF000AC037091AD03A091AF03B091B003C62F96
:103F0000C72316E0D81304C0DF91CF911F91089505
:103F100090E0109711F0CF3F19F401968770F2CF1F
:103F2000189F9001199F300D1124F901ED54FC4F99
:103F300041814713F2CF40814613EFCF42814111B7
:103F4000ECCF438154814A1B5B0B483C510528F759
:103F50008091B1038F7080618093B103F901E854BF
:103F6000FC4F80818F70806180838CEA93E00E9497
:103F70000119DF91CF911F910C948F06AF92BF92E0
:103F8000CF92DF92EF92FF920F931F93CF93DF9325
:103F9000CDB7DEB761970FB6F894DEBF0FBECDBFC9
:103FA0008C0185E0F801DE011D9601900D928A9545
:103FB000E1F7F80180819181E2802CEAA22E23E0D2
:103FC000B22E6091AF037091B0036115710509F4D1
:103FD0003EC13091AC034091AD03232F24232F3FEA
:103FE00009F435C1C380D480F090AE03F601E61B1E
:103FF000F70BFF2009F4FBC02091B103522F507F33
:10400000E83CF10508F0BBC0511178C0FE2C491303
:1040100021C038131FC0E1101DC02F7020612093F4
:10402000B103C5010E9401198091B103F801858394
:104030008F2D61960FB6F894DEBF0FBECDBFDF9116
:10404000CF911F910F91FF90EF90DF90CF90BF9095
:10405000AF900895CD2829F0282F29232F3F09F06C
:1040600014C120E0F22FF170DF2E20FF3DC020911F
:10407000E3034091B20356E0241315C08D879E8759
:104080008D859E850E94D40C292F22952F70223079
:10409000F8F0243020F59F70F9F0F8019581907FB9
:1040A000D9F4D12C1FC030E0529FF001539FF00D86
:1040B0001124ED54FC4F6181961306C06081861374
:1040C00003C06281E61210C02F5F3F4F2770D4CF2C
:1040D0009F7011F0882329F3805E883010F3C801A7
:1040E0000E940119FD2CA4CFEE2009F4A1CF8091EC
:1040F000B10381608093B103F12C9ACF491312C0B0
:10410000381310C0E1100EC0F8012583C8010E94C9
:10411000011986E0F801ACEAB3E001900D928A95AE
:10412000E1F786CF8D879E878D859E850E94DE0C68
:10413000882309F1EE20F9F08091B103803270F00C
:104140002091AC033091AD0338872F831986DB862D
:10415000CA868C87CE0107960E94011986E0F80175
:10416000ACEAB3E001900D928A95E1F70E94681FD6
:10417000FF24F3945DCFC8010E940119F9CF5111BA
:104180000AC08CEA93E00E94011986E0F5011192C1
:104190008A95E9F7B1CF49130FC038130DC0E1106C
:1041A0000BC0F8012583C8010E94011986E0F501C2
:1041B00011928A95E9F73CCF8D879E878D859E85E4
:1041C0000E94DE0C8823B9F2EE20A9F28091B1039F
:1041D000803220F22091AC033091AD033A832983E1
:1041E0001B82DD82CC828E83CE010196B5CFE83C66
:1041F000F105E0F6FE2CEE2009F4BDCF491316C000
:10420000381314C08091B10380FD83CF982F907F25
:1042100009F47FCFF8018583903F09F477CF982F79
:10422000907F905F8F70892B858370CF8D879E875D
:104230008D859E850E94DE0C811190CF8091B10307
:1042400081608093B103C8010E940119F1CEEE2074
:1042500009F491CF8D879E878D859E850E94DE0C07
:10426000F82E882309F487CF86E0F801ACEAB3E0A2
:1042700001900D928A95E1F78091AC039091AD0386
:104280000E94D40C0E94681FD3CE21E02E25EACED6
:104290001F93CF93DF93CDB7DEB767970FB6F89430
:1042A000DEBF0FBECDBF342F4B8B252F5C8B6D8BAC
:1042B0007E8B8F8B8E899F896111109222041A8ABE
:1042C000198A3D872E876F87998B888B86E0FE0140
:1042D0003D96DE01179601900D928A95E1F7CE0189
:1042E00007960E94BE1F882389F016E08091E303A1
:1042F0009091B203891349C067960FB6F894DEBF58
:104300000FBECDBFDF91CF911F91089586E0FE01D2
:104310003796DE01119601900D928A95E1F78A8514
:104320009B85892B11F38F81988589238F3FE9F233
:104330002091B20330E0C90101968770992740911E
:10434000E3034817190671F40E94B7151092B203DF
:104350001092E30386E0ECEAF3E0DF011D928A9518
:10436000E9F7C3CF96E0929FD001939FB00D11243F
:10437000AD54BC4FFE01319601900D929A95E1F734
:104380008093B2030E948F06B0CF819FC001112499
:104390008D549C4F0E94BE1F882309F4ADCF80919D
:1043A000E30390E00196877099278093E3039ECF03
:1043B0001F920F920FB60F9211242F933F934F939A
:1043C0005F936F937F938F939F93AF93BF93CF939D
:1043D000DF93EF93FF93D091E900DF708091EC00C1
:1043E000C82FC17080FDC0E81092E9008091F000F4
:1043F000877F8093F00078940E94CC151092E9009A
:104400008091F00088608093F000CD2BCF70C09336
:10441000E900FF91EF91DF91CF91BF91AF919F9113
:104420008F917F916F915F914F913F912F910F905D
:104430000FBE0F901F9018951F920F920FB60F92FC
:1044400011242F933F934F935F936F937F938F9399
:104450009F93AF93BF93EF93FF938091E10082FF0F
:1044600009C08091E20082FF05C08091E1008B7F4E
:104470008093E1008091DA0080FF24C08091D80011
:1044800080FF20C08091DA008E7F8093DA008091D7
:10449000D90080FF9BC080E189BD82E189BD09B45C
:1044A00000FEFDCF81E08093980480917304811118
:1044B00009C00E94E6030E94B1048091E20084607A
:1044C0008093E2008091E10080FF17C08091E200BC
:1044D00080FF13C08091E2008E7F8093E200809184
:1044E000E20080618093E2008091D8008062809336
:1044F000D80019BC85E0809398048091E10084FF86
:1045000029C08091E20084FF25C080E189BD82E15D
:1045100089BD89B5982F917080FFFBCF8091D8001D
:104520008F7D8093D8008091E1008F7E8093E100A1
:104530008091E2008F7E8093E2008091E2008160B2
:104540008093E20080919904882309F445C084E0B7
:10455000809398048091E10083FF27C08091E2005E
:1045600083FF23C08091E100877F8093E10082E098
:1045700080939804109299048091E1008E7F80933B
:10458000E1008091E2008E7F8093E2008091E20062
:1045900080618093E20042E060E080E00E947F045E
:1045A0008091F00088608093F000FF91EF91BF91BF
:1045B000AF919F918F917F916F915F914F913F91BB
:1045C0002F910F900FBE0F901F90189519BC10924D
:1045D00098041092730476CF8091E30087FD93E0F6
:1045E00090939804B7CFCDB7DEB7AA970FB6F894DB
:1045F000DEBF0FBECDBF84B7877F84BF0FB6F894F0
:10460000A89580916000886180936000109260009E
:104610000FBE80E890E00FB6F8948093610090930D
:1046200061000FBE85B7806885BF85B7806885BF8C
:1046300081E795E090939F0180939E010E94E6039D
:104640000E94B1048091E20084608093E20078943B
:10465000809198048823A1F01091E9001F70909137
:10466000EC00892F817090FD80E8182B1092E900F2
:104670008091E80083FD0E94CC151F701093E90023
:1046800082E084BD93E095BD9AEF97BD80936E0064
:1046900009E711E0E8E8EE2EE1E0FE2EF801819155
:1046A0008F010E94640AE016F106C1F786E60E94B7
:1046B000640A80E30E94640A81E30E94640A82E340
:1046C0000E94640A83E30E94640A87E30E94640AEA
:1046D000E9E2F4E085E394E0A3E6B4E011921192FC
:1046E0001D921D928E179F07C9F70E94D811FFEFE8
:1046F00026E741E0F15020404040E1F700C00000D3
:104700000E94D8118091630480FF17C06FEF82E28E
:1047100090E00E94E9296FEF83E290E00E94E9298E
:104720006FEF84E290E00E94E9296FEF7FEF90E065
:1047300080E00E94072A0E94130E0E940914811132
:1047400002C00E941414269A2E9882E28093800060
:1047500089E1809381008FEF9FEF90938700809392
:1047600086000E947E1482E290E00E94D529813268
:1047700009F0CDC483E290E00E94D529873009F08A
:10478000C6C484E290E00E94D529823109F0BFC4FA
:104790000E940914811102C00E94141482E090E06A
:1047A0000E94D52980934E040E94BE0A909336043D
:1047B0008093350483E090E00E94D529682F70E053
:1047C00090E080E00E94D0080E947E14809137041F
:1047D000811133C00E940914811104C00E94141475
:1047E0000E94A71588E090E00E94DD2960935E0496
:1047F00070935F0480936004909361046E7F71F402
:104800000E94A71588E090E00E94DD2960935E0475
:1048100070935F0480936004909361040E945B072F
:1048200010925D0480915E0480FF04C060E0869574
:104830000E949E1881E08093370482E191E090937A
:1048400039048093380458E1E52EF12C60E4B62E4B
:104850007FE6C72E74E0D72E8091980400E112E124
:10486000853009F4BCC10E94D811882359F08FB754
:10487000F89440916F0450917004609171047091AC
:1048800072048FBFEFE4F4E0A3E6B4E010E000E0D0
:10489000702F8D919D91219131912817390709F43D
:1048A000B0C12827392760E088248394912CA9017E
:1048B00048215921452B09F49EC169A37AA39C0183
:1048C0002821392191E0232B09F490E09BA30E9439
:1048D00085058160782F9DA38CA349A15AA16BA166
:1048E0008DA10E944821000F111FF801E15BFB4FD1
:1048F00080819181882699269182808280915D04B1
:104900008823D1F180915C04E0915E04E695E81B78
:10491000E0933D04823009F08BC1F0E0E455F94F9B
:10492000E4910E2F10E0F4EB8F2EF1E19F2E809199
:104930003E04882361F010923E040E948505909306
:104940003C0480933B041092400410923F040E9468
:104950008505E0913B04F0913C048E1B9F0B8F3F3B
:104960009F4750F4E00FF11FF0933C04E0933B04A9
:104970008BE394E0F401099586E0E7E4F4E0DE01DE
:10498000119601900D928A95E1F7909049048090DC
:104990004A0410914B0400914C0410924904109267
:1049A0004A0410924B0410924C04892D882909F472
:1049B00048C080914504909146040E9476059C0170
:1049C00090914404992309F4C9C323333105C8F1F4
:1049D0009F3F19F09F5F90934404992059F00E94E3
:1049E000DC099FEF19140CF491E0899F802D1124AC
:1049F00080934904882059F00E94DC099FEF181425
:104A00000CF491E0899F802D112480934A04309109
:104A100049043323B1F020914A04222391F045EB5D
:104A20003403C0011124992309F46EC19093490401
:104A300045EB240390011124332309F469C1309319
:104A40004A04812F802B09F448C080914204909140
:104A500043040E9476059C0190914104992309F436
:104A600078C325363105C8F19F3F19F09F5F9093B9
:104A70004104112359F00E94BA099FEF11160CF45A
:104A800091E0899F802D112480934B04002359F0DD
:104A90000E94BA099FEF10160CF491E0899F802DB7
:104AA000112480934C0430914B043323B1F02091B6
:104AB0004C04222391F045EB3403C00111249923C7
:104AC00009F42AC190934B0445EB2403900111246F
:104AD000332309F425C130934C048091490490910B
:104AE0004A04892B90914B04892B90914C04892B7B
:104AF00011F00E940A0886E0FE013196A7E4B4E0B6
:104B000001900D928A95E1F70E94DA0690914D048A
:104B1000891721F00E94DA0680934D048091980451
:104B2000843009F099CE83E08093E9008091E80019
:104B300082FF92CE8091E80090E085FF06C00E943F
:104B40000504882309F4F0C091E08091E8008B7798
:104B50008093E800992309F47FCEE981E150E331A5
:104B600008F064C1F0E0E654F54D0C9450298091B2
:104B70009804843021F180E00E94E60610923A0405
:104B80000FB6F894A895E09260000FBEB092600056
:104B900083B7817F846083BF83B7816083BF78944C
:104BA000889583B78E7F83BF0FB6F894A8958091C0
:104BB0006000886180936000109260000FBE809159
:104BC0009704882361F00E94D811E3E6F4E0819114
:104BD0009191892B09F085C2CE16DF06C1F780912D
:104BE0009804853009F4C3CF0E94B7150E947E1443
:104BF0000E94DA0638CE6F5F880C991C6F3009F07E
:104C000056CE0F5F1F4F0630110509F041CE8FEFD2
:104C10008EA38FA318A60E9485058160782F9AA77E
:104C200089A74EA15FA168A58AA50E94482166CEEA
:104C3000863059F4F0E0E755F94FE4910E2F10E07B
:104C4000E8EC8E2EE1E19E2E72CE893061F4E6957D
:104C5000F0E0EA55F94FE4910E2F10E072EA872E4A
:104C60007FE0972E64CE8F3061F4E695F0E0ED554D
:104C7000F94FE4910E2F10E06CEC862E6FE0962E2B
:104C800056CE853159F4F0E0E056F94FE4910E2FFD
:104C900010E05AE3852E50E1952E49CE08E210E04F
:104CA00028E8822E20E1922E883109F440CE83320A
:104CB00049F4EEE9F6E0059114914BE5842E41E1CB
:104CC000942E35CE04EF11E091E1892E91E1992ED9
:104CD000843209F42CCE853281F48E2F63E00E9459
:104CE0000E29E92FF0E0E556F94FE4910E2F10E080
:104CF0003AE5832E33E1932E1ACE00ED17E080E7DC
:104D0000882E85E0982E13CE81E08093490490CEC2
:104D100081E080934A0495CE81E080934B04D4CE09
:104D200081E080934C04D9CE00E210E0CE010196E0
:104D30004C018091E80085FD0AC08091E8008B77E6
:104D40008093E8000E940504882399F3FDCE8091AA
:104D5000F100F40181934F010150110951F7F4CE94
:104D60001A8289E08B831AC08A81823009F4E8C1F3
:104D70008330D9F1813009F059C02FB7F894609190
:104D80006F047091700480917104909172042FBF30
:104D90000E9456296B837C838D839E838091980427
:104DA000843009F059CD1091E9001F709091EC000A
:104DB000892F817090FD80E8182B82E08093E900B4
:104DC0008091E80080FF0DC050E040E060E270E0BC
:104DD000CE0101960E9436048091E8008E77809380
:104DE000E8001F701093E90037CDDE011196E3E66D
:104DF000F4E080819181329612969C9312971396DB
:104E00008C931397129624E0EF36F20791F7C6CFF2
:104E10008A81823059F46B817C818D819E810E94D0
:104E2000562985E290E00E94E929B8CF8FEF898367
:104E3000B5CF4C816B818A810E94CC0A9827892743
:104E400098279E838D83AACF2D813E8132272327E9
:104E500032274C816B818A810E94170D9FCF0E945F
:104E6000400D9CCF8A81893061F48B8143E0849F1F
:104E7000C00111246FEF70E00E942829862F0E9444
:104E800040078A818138C1F060F4803809F086CF0C
:104E900020E04B816091600480915F040E94AE1419
:104EA0007DCF823859F1833809F078CF20E04091E6
:104EB00061046C818B81F2CF60E08B810E949E182F
:104EC0009B8180915E04911111C08E7F80935E045E
:104ED00010925D048FEF90E7E2E081509040E04057
:104EE000E1F700C000000E946D0F58CF81608093F1
:104EF0005E0460E086950E949E1850CF8B8180935F
:104F000062044CCF8A81893059F08A30C1F08138EF
:104F100021F1B8F4803809F041CF8091610422CFAB
:104F200080915B04869586958695FFEF8F9FC001E3
:104F3000112463E070E00E9428296B832FCF1B822D
:104F40002DCF823891F0833809F028CF80915F040B
:104F50008B83809160048C8321CF80915E0480FFDD
:104F600002C08695FFCE80E0FDCE80916204FACE2D
:104F700080915B040E94020D60915E0470915F0459
:104F800080916004909161040E949C1407CF80E19D
:104F90008A8304CF81E08A838AE0E4CE0C8110E02A
:104FA0000D31110508F0FACE8A809B80982489245F
:104FB0009824CE0101963C01080F191FC4018A50A4
:104FC0009D4F6016710609F4E9CEFAE08F16F1E004
:104FD0009F0658F40E94D529F3018483FFEF8F1AAE
:104FE0009F0A2FEF621A720AE9CFF3011482F6CFFB
:104FF0008C80912C4DE18416910408F0CFCE0A816B
:105000001B81102701271027CE0101963C01800E3D
:10501000911EC8018A509D4F8016910609F4BECE9C
:105020000A30E1E01E0720F4F30164810E94E929BF
:10503000FFEF6F1A7F0A0F5F1F4FEBCF0E94070D24
:10504000ADCE84E0A5CF0C8110E00D31110508F044
:10505000A5CE8A809B80982489249824CE0101962D
:105060003C01080F191FC40186960615170509F49F
:1050700095CEF0ED8F16F2E09F0658F40E94D529E8
:10508000F3018483FFEF8F1A9F0A2FEF621A720ACF
:10509000EACFF3011482F6CF8C80912C4DE1841677
:1050A000910408F07BCE0A811B811027012710276D
:1050B000CE0101963C01800E911EC8018696801695
:1050C000910609F46BCE003DE2E01E0720F4F301E7
:1050D00064810E94E929FFEF6F1A7F0A0F5F1F4F5B
:1050E000ECCF09BD19BD09B400FEFDCF8091D800F9
:1050F0008F7D8093D8008091E00082608093E000F3
:105100008091E00081FDFCCF0E94B71568CD60E082
:1051100085E290E00E94E9290E94400D0E94070D5F
:1051200061E282E290E00E94E92967E083E290E098
:105130000E94E92962E184E290E00E94E92928CBFB
:1051400085E290E00E94D5291B821C821D828E83FD
:1051500025CE2D32314008F089CCBFCC2D323140E4
:1051600008F038CC6ECC78941F921FB61F92112491
:105170008F939F93AF93BF9380916F04909170042E
:10518000A0917104B09172040196A11DB11D80938C
:105190006F0490937004A0937104B0937204BF9154
:1051A000AF919F918F911F901FBE1F9018951F92D6
:1051B0001FB61F9211248F939F93AF93BF9380913B
:1051C0003A04811113C080916F0490917004A091F2
:1051D0007104B09172044196A11DB11D80936F04BA
:1051E00090937004A0937104B0937204BF91AF9137
:1051F0009F918F911F901FBE1F901895DB018F9379
:105200009F930E943C2ABF91AF91A29F800D911D58
:10521000A39F900DB29F900D11240895991B79E0E2
:1052200004C0991F961708F0961B881F7A95C9F736
:105230008095089587FB082E062687FD819567FDDA
:1052400061950E940E290EF4919507FC81950895B1
:10525000AA1BBB1B51E107C0AA1FBB1FA617B7079C
:1052600010F0A61BB70B881F991F5A95A9F78095B8
:105270009095BC01CD01089597FB072E16F400947C
:1052800007D077FD09D00E94282907FC05D03EF4FD
:10529000909581959F4F0895709561957F4F0895E2
:1052A000EE0FFF1F0590F491E02D099469279627D2
:1052B000692778278727782708950E94712A332342
:1052C00012F48A1B9B0B0C9467290E94712AB7FF6A
:1052D0000895821B930B08958F929F92AF92BF9275
:1052E000CF92DF92EF92FF92CF93DF93EC01688130
:1052F00079818A819B81611571058105910521F470
:1053000064E279ED8BE597E02DE133EF41E050E089
:105310000E941D2A49015A019B01AC01A7EAB1E490
:105320000E943C2A6B017C01ACEEB4EFA501940114
:105330000E944A2ADC01CB018C0D9D1DAE1DBF1DB4
:10534000B7FF03C00197A109B04888839983AA8356
:10535000BB839F77DF91CF91FF90EF90DF90CF904D
:10536000BF90AF909F908F9008950E946C290895F0
:1053700080E091E00E946C290895B0E0A0E0809365
:10538000000190930101A0930201B09303010895DD
:10539000FC014150504030F001900616D1F7319792
:1053A000CF010895882799270895F999FECF92BDD6
:1053B00081BDF89A992780B50895A6E1B0E044E050
:1053C00050E00C940F2AA8E1B0E042E050E00C94C9
:1053D0000F2A262FF999FECF92BD81BDF89A019729
:1053E00000B4021639F01FBA20BD0FB6F894FA9A2D
:1053F000F99A0FBE08950396272F0E94EA290E946A
:10540000E929252F0E94EA29242F0C94EA290196E4
:10541000272F0E94EA290C94E929DC01CB01FC0129
:10542000F999FECF06C0F2BDE1BDF89A319600B4FD
:105430000D9241505040B8F70895052E97FB1EF489
:1054400000940E94342A57FD07D00E944F2A07FC7F
:1054500003D04EF40C94342A509540953095219504
:105460003F4F4F4F5F4F0895909580957095619590
:105470007F4F8F4F9F4F08950E94712AA59F900DD7
:10548000B49F900DA49F800D911D11240895B7FF26
:105490000C943C2A0E943C2A821B930B0895A1E2A3
:1054A0001A2EAA1BBB1BFD010DC0AA1FBB1FEE1F9E
:1054B000FF1FA217B307E407F50720F0A21BB30BE9
:1054C000E40BF50B661F771F881F991F1A9469F765
:1054D00060957095809590959B01AC01BD01CF01C1
:1054E0000895A29FB001B39FC001A39F700D811DBD
:1054F0001124911DB29F700D811D1124911D0895DD
:10550000F894FFCFED0CED0CF60CF60CF80CF60C45
:10551000F60CF60CED0CED0CFD0CF60CF60CFD0C7F
:10552000B116D9162C17D9162C170C1744172C178F
:105530004C185918391C391C951C951CEE1C081D5B
:105540006E1C6E1C151DEB1DFA1DFA1D621B891BBE
:10555000901B951B9A1B9F1BA41BA91BAE1BB31B67
:10556000B81BBD1BC01BC51BC81BCB1BCE1BD11B37
:10557000D41BD71BB026B4260827192724272F278A
:1055800032278227B82716271627C727CA27CE27EC
:0A559000F8271E28212823284C28A4
:10559A000100000001191A1B1C1D1E1F20212201D7
:1055AA0002017305D30DB20DAE0DAA0D0100010261
:1055BA000202020606060909090909090F0F0F0F57
:1055CA000F0F151515181919191919191919191962
:1055DA002324252525252525818283E200E900EA61
:1055EA0000B500B600B700CD008301CC008A019255
:1055FA000194012102230224022502260227022AFB
:10560A0002B300B4006F0070009091929395949643
:10561A009734F7F6F5F4F1F0663031323337402239
:0E562A00BC8A016801AC00C206DB06FB06006C
:00000001FF
